:1000000083168511860183128C018C0A8C0A7F303D
:100010008600851150308F0005190A288F0B0C2897
:1000200050308F009100900004308D0002300C069B
:10003000031D1C2885111D2885150C0865208600C8
:100040008C0803190A2808300C0603190A280D0821
:100050008E0005080739920012193028121532282F
:1000600012110000121D70208F0B39280E15503010
:100070008F00921C7820900B40288E1450309000F6
:10008000121C7420910B47280E14503091000E085A
:100090000D06031927280E088D000E0803192728BE
:1000A0000E1D552802308C0016288E1C5E288C0AE6
:1000B00002300C06031D16288C0A16288C03023009
:1000C0000C06031D16288C03162882076734F634A5
:1000D00084344C3454343634153405343E346F286B
:1000E0000E1150308F0008000E10503091000800A3
:0800F0008E1050309000080052
:02400E00FB3F76
:00000001FF
